:10002200F894AA27ACBBA8E1A1BDA0E1A1BDAA2773
:10003200A5BF0024A0E6BB27C0E0D1E00D92219726
:10004200E9F7EEE6F1E0C895102C3196C8953196A5
:10005200CE2FDF2FF02DE12D3097A1F0C895A02DE6
:100062003196C895B02D3196C895802D3196C89598
:10007200902D3196C8950D9231960197D9F7EC2FB4
:10008200FD2FE1CFAFE5B1E0ADBFBEBFCFE9D0E01C
:10009200A3E3A9B94CC0E8B7AE2FE1E0EA23EE230F
:1000A20009F001C0F8CFE5EBE2BFE8B7AE2FE1E01F
:1000B200EA2BE8BF0895E091A000EF5FE093A00073
:1000C200E150E091A000AE2FE4E657D0EE2309F410
:1000D2001AC0E5B3AE2FE0E8EA27E5BBEE27E093CE
:1000E200A000E091A100AE2FE1E0EA27E093A10099
:1000F200EE2720FCE1E0AE2FE1E0EA27E8940024BD
:10010200E011689420F80895EEE1E5BD0895EEE26D
:10011200E5BD0895EE2720FCE1E0AE2FE1E028D016
:10012200EE2309F402C0F0DF01C0F1DF0895EE27EB
:10013200EABBEFEFE7BBEFEFE4BBE0E8E1BBEE27A2
:10014200E8BBEE27E5BBEE27E093A100E1E0E9BFC3
:10015200E5E0E3BFE7E2E3BDEFE1E5BD9CDFD4DF2D
:10016200AADFFCCF0895020002000000680100002F
:10017200EA17E1E009F0EE270895EA17E1E008F056
:04018200EE270895C7
:1000000010C0FECFFDCFFCCFFBCFFACFF9CFF8CF9A
:10001000F7CFF6CFF5CFF4CFF3CFF2CFF1CFF0CFCC
:02002000EFCF20
:00000001FF
